:020000040000FA
:04000000FA3060284A
:080008008612601C8616BA0086
:10001000030EBB008312051E21285008E000510882
:10002000E1005208E2005308E3005408E4005508D8
:10003000E5005608E6005708E700601C86166018C1
:100040008612051921280F30A9008B100314851E74
:100050000310C01BE70C401BE60CC01AE50C401A4D
:10006000E40CC019E30C4019E20CC018E10C401874
:0C007000E00C3B0E8300BA0E3A0E0900B3
:1000C000203084008001840A80300402031C6228EE
:1000D0008316FF3085051F308605C73087058312DC
:1000E000850186018701103083168E0083127030DF
:1000F00083168F008312003003179900031300301A
:1001000003179A0003130030970000309F0000305F
:1001100083169F008312003003179E0003130030E4
:1001200003179F000313C7308316810083123030FA
:10013000900000309200003083169400831200304B
:100140009400A630831698008312003083169B001B
:1001500083120030980033308316990083120030E8
:1001600083168C008312003083168D0083121030AA
:100170008B00C20BB9280130AA0081018E018F01CA
:100180000B118B100B108C128C018D018B176400DE
:100190000B19CC20DC20C7280B11AA0B0800043057
:1001A000AA000021A9080319D8280613A9030800EA
:1001B0000609403986000800031087180314C80D8B
:1001C00048120C304802031D0800C801061EF5281D
:1001D0004E08031DF32841180821C1180F214119A9
:1001E0001821C1192F212030CE00CE03031007198A
:1001F0000314CD0CCC0CCB0CCA0C08004314080023
:100200000130871F0430C1000310071FC10D080013
:100210000330C0004A08D0004B0AD1000800073064
:10022000C0004A08D0004B0AD1004D08D200080097
:100230000F30C0004A08D0004B0AC200D801D901D3
:10024000DA010314D80DD90DDA0D0310C20B2229DF
:100250005808D1005908D2005A08D3000800FF30CE
:10026000C0004A08D0004B0AC200D801D901DA0107
:100270000314D80DD90DDA0D0310C20B39294D081E
:10028000D700CA1F4D29D101D201D3015808D4008B
:100290005908D5005A08D6000800D401D501D60166
:1002A0005808D1005908D2005A08D300080007089E
:1002B000203A870008000708103A8700080007085E
:0602C000083A8700080067
:084000000800000000000400AC
:02400E00CC03E1
:00000001FF
